:1000000043288316051485108312080090000A30D7
:100010008F00031003188510031C8514AA308E006E
:100020008E0B10280314900C8F0B0A280800101058
:10003000051C003409308F0038308E008E0B1E28CE
:100040000310051C0314900CAA308E008E0B26287A
:10005000000000008F0B2028100810140800B13099
:100060008C0003308D008C0B33288D0B3328080057
:1000700006143D2006103D20080000008C0B3D2892
:100080008D0B3D28080001208316051186120610ED
:1000900083120511382038203820051A5228061EF0
:1000A00055285D28061E62286C28061405111720A5
:1000B000101C4D28013E06204D28061020308606D3
:1000C0002F2078288616013086063D20910A1108D7
:1000D0000F39413E06207828013086063D203D201C
:1000E0003D203D208612910A11080F39613E0620FD
:0400F00005154D287D
:02400E00F23F7F
:00000001FF
